:10250A00C10A4202A4000444026E00000000440210
:10251A0072000000004402760000000044027A00C3
:10252A0000000044027E0000000044028200000015
:10253A00004402860000000044028A0000000042B3
:04254A00028E000AF3
:101796001211819002D4E47FFF7E03FDFC0211400A
:1017A600C374FF9BFB74039AFAE499F9E498F8E48E
:1017B600FCFD120FD3780A02110E1211409002E8B6
:1017C600C374FF9BFF74039AFEE499FDE498FC0240
:1017D60011819002D8E47FFF7E03FDFC021140E4F4
:1017E600FCFD120FD39002DC1211819002DC021173
:1017F60034E4FCFD120FD39002E01211819002E056
:10180600021134AE18AF199002D8E4FCFD02114063
:10181600121134EF24FCFFEE34FFFEED34FFFDEC35
:1018260034FFFC22E47FFF7E03FDFC121140D3024D
:1018360010FD121134EF2404FFE43EFEE43DFDE406
:101846003CFC22E47FFF7E03FDFC121140C3021024
:10185600FD9002D4121134780A021121AE10AF1194
:10186600AB07AA06E4F9F822780A12110E9002E0F4
:10187600021181900346E0FFA3E0FDA3E0FB229066
:1018860002A9E0FF900345E06F2212105E9002DC91
:1018960002118112105E9002E402118112105E9014
:1018A60002E8021181121140C374FF9BFB74039A74
:1018B600FAE499F9E498F822ADBBED25E0244EF858
:1018C600A60608A6072290027A1211349002D422A4
:1018D60090028A1211349002D8229002E802114036
:1018E6009002E4021140C374FF9511FF7403951032
:1018F60022C374FF9519FF7403951822900296E48B
:10190600F0A322900298E4F0A32290029CE4F0A3B4
:101916002290029AE4F0A3229002D0021140900293
:10192600D40211349002D8021134E4FCFD9002D4A2
:10193600229002E8021134C3E51194FFE5109403E6
:10194600229002E4021134C3E51994FFE5189403CA
:01195600226E
:1026B300900208E0FEA3E0FF900204E0FCA3E0FD2B
:1026C300B50719ECB5061590020CE0FEA3E0FFED8B
:0E26D300B50709ECB5060520C502D322C322C7
:1028620075F1FEE4F5F2F5F375A41A75D41175E16C
:052872000675E2C02222
:1028DE0075D10275BC4075E8C075BA1F43F6084342
:0328EE00E60822D7
:0F29040075A14075F80175A20243B840D2AE220A
:091A2400E4F5B1F5A975B28322C5
:0B292C0075CA8275CBFDD2CAD2AD2265
:0D2913007592077593F875910443E68022D4
:10283400E4F5D9121A241228621228DE122904128D
:08284400264F12292C02291372
:0B293700E5B030E403C20D22D20D22F7
:08294B0090035BEFF0021A1B80
:0829530090035BEFF002284C39
:08294200E4FFE5B030E3010FF2
:01294A00226A
:1027A700EF25E0FFA20DE4334F14601314600A1401
:1027B700600A240370097F36227F37227F35227F04
:0227C7003422BA
:10121000E4FDFF12150F7D017F0112150F7D027F86
:101220000212150F7D037F0312150F7D0A7F041232
:10123000150F7D0B7F0512150F7D0C7F0612150F04
:101240007D0D7F0712150F7D0E7F0812150F7D0F84
:101250007F0912150FD3E5139430E512940340086B
:101260001219027410F08040D3E5139464E51294CF
:101270000240081219027408F0802DD3E5139498E7
:10128000E512940140081219027404F0801AD3E5A3
:101290001394CCE5129400900296E44007F0A374F6
:1012A00002F08004F0A304F0D3E50F9430E50E942F
:1012B0000340081219097410F08040D3E50F9464BC
:1012C000E50E940240081219097408F0802DD3E548
:1012D0000F9498E50E940140081219097404F080E7
:1012E0001AD3E50F94CCE50E9400900298E44007E1
:1012F000F0A37402F08004F0A304F0D3E50B943063
:10130000E50A9403400812191074D0F08041D3E527
:101310000B9464E50A9402400812191074C8F08016
:101320002ED3E50B9498E50A940140081219107425
:10133000C4F0801BD3E50B94CCE50A940090029C8A
:10134000E44007F0A374C2F08005F0A374C1F0D3A9
:10135000E51B9430E51A9403400812191774D0F075
:101360008041D3E51B9464E51A94024008121917D2
:1013700074C8F0802ED3E51B9498E51A94014008B8
:1013800012191774C4F0801BD3E51B94CCE51A9492
:101390000090029AE44007F0A374C2F08005F0A325
:1013A00074C1F0E5097003021452D3E5179430E5D7
:1013B00016940340089002A37410F0803CD3E51704
:1013C0009464E516940240089002A37408F0802902
:1013D000D3E5179498E516940140089002A374048D
:1013E000F08016D3E51794CCE51694009002A34044
:1013F000057402F080037401F0D3E5119414E51034
:10140000940340089002A3E044A0803BD3E51194EC
:1014100054E510940240089002A3E044808028D351
:10142000E51194A4E510940140089002A3E0446003
:101430008015D3E51194ECE51094009002A3E040F0
:1014400004444080024420FF9002A0E4F0A3EFF0A7
:101450008007E49002A0F0A3F0E5087003021507EE
:10146000D3E51D9430E51C940340089002A374104A
:10147000F0803CD3E51D9464E51C94024008900282
:10148000A37408F08029D3E51D9498E51C940140CD
:10149000089002A37404F08016D3E51D94CCE51CDB
:1014A00094009002A340057402F080037401F0D30D
:1014B000E5199414E518940340089002A3E044A0B1
:1014C000803BD3E5199454E518940240089002A398
:1014D000E044808028D3E51994A4E51894014008DD
:1014E0009002A3E044608015D3E51994ECE51894CC
:1014F000009002A3E04004444080024420FF900298
:0F1500009EE4F0A3EFF022E490029EF0A3F0220D
:101BCF001228341229427572077524077525D01211
:101BDF0029371227A79002A9EFF0300D0543A480F3
:101BEF00C287D2AF43E60112280212284CE56F607C
:101BFF003614601414600924FE70296309018003F0
:101C0F006308011228F1801C300A0F300D05A287DE
:101C1F00B3928730870EC218800AE4FF12294B3027
:101C2F000D02C287E4F56F300E13C20EE525452471
:101C3F006008E5251525700215241212101226834F
:101C4F00EF60AA900344E0FFB40B02D20AEF6431B5
:101C5F00702612188570211226B350FB121D5412D4
:101C6F0026B350FB121879A3E0900305F012202041
:101C7F001226B350FB121D5D900344E064327020B6
:101C8F00121885701B1226B350FB121D541226B367
:101C9F0050FB1218791220EF1226B350FB121D5D64
:101CAF00900344E0642D702A12188570251226B314
:101CBF0050FB9002A9E0FF1228A11226B350FB128D
:101CCF0018791221B91226B350FB9002A9E0FF1226
:101CDF00288C900344E0642E702A12188570251208
:101CEF0026B350FB9002A9E0FF1228A11226B35091
:101CFF00FB1218791222491226B350FB9002A9E069
:101D0F00FF12288C30871C900344E014600D047080
:101D1F0012900345E0FF1229538008900345E0FF1E
:101D2F0012294B900344E0FFB41407300D04D287FF
:101D3F00C218EF64156003021BFC200D03021BFC8D
:051D4F00C287021BFC2D
:101D54009002A9E0FF1228A1229002A9E0FF122814
:021D64008C22CF
:10235900E5B05407F56E6572600CE56E6572F5704F
:10236900757103856E72E57160361571E5717030AE
:10237900E57030E211E56E20E20C9002A77405F0D9
:10238900A374DCF0D20BE57030E108E56E20E103BF
:10239900756F02E57030E008E56E20E003756F01A6
:1023A900300B2B9002A774FFF5F0120F8CE5B05497
:1023B900046005756F04C20B9002A7E07002A3E0E8
:0E23C900700CC20B9002A9E0FF7D071219F202
:0123D70022E3
:031A12000208A720
:1008A700C0E0C0F0C083C082C0D075D000C000C017
:0D08B70001C002C003C004C005C006C00798
:1008C400C2CF9002A2E4F0900290A3E0F5A39002BC
:1008D400A4E4F0A37404F0F5BB75E8D02009030286
:1008E4000E50E50D2559FFE50C3558FEE4FCFD904E
:1008F40002CC121181E515255FFFE514355EFEE497
:10090400FCFD9002D01211819002CC12179CD312DC
:1009140010FD400A9002CC12118D000003FF9002DA
:10092400D01217DBD31210FD400A9002D012118DA1
:10093400000003FF9002CC121140AE56AF571217BD
:10094400A6C004C005C006C007AE5AAF5B9002CC77
:100954001218101217B8D003D002D001D000120F11
:10096400B89002D412118112191EAE5CAF5D121739
:10097400A6C004C005C006C007AE60AF61E4FCFDBC
:1009840012191E1217B8D003D002D001D000120FD2
:10099400B89002D81211819002721218CF12183135
:1009A40040141219249002721211819002D4121868
:1009B4001690027A801A1218CC1218505015121977
:1009C4002490027A1211819002D412183890027283
:1009D4001211819002821218D9121831401412197E
:1009E4002A9002821211819002D812181690028A5B
:1009F400801A1218D6121850501512192A90028A09
:100A04001211819002D812183890028212118112A8
:100A140018CC1211811218D6121796D31210FD4059
:100A24000A9002D412118D000003FF1217D8D312BA
:100A340010FD400A9002D812118D000003FFE50951
:100A44007003020B81AE54AF551219301218505076
:100A5400611218571217EBC006C007121862D007AC
:100A6400D0061218909002DC121140AE16AF171285
:100A740017E5780A12110E1218931218571218A5B6
:100A8400121937C006C007121862D007D006121810
:100A9400A29002E81218499002E850051217C0808B
:100AA4000712118D000000001218E0AE0EAF0F0205
:100AB4000B65AE10AF11121930121831400E121816
:100AC40062121924120FC5121893800A9002DC12C4
:100AD400118D000000001217F1780A12112112186A
:100AE4009312193D50151218ECFEE4FCFD9002E837
:100AF4001217EE1218E0121890800A9002E81211F0
:100B04008D000000009002DC121140AE0AAF0B12FF
:100B140017E5780A12110E9002DC121796C3121010
:100B2400FD50089002D41217C0800A9002E81211F6
:100B34008D000000009002E812185A1218A512192C
:100B44003D5017121937C006C0071218ECAB07FA4C
:100B5400E4F9F8D007D0061218A21218E0AE16AFC6
:100B640017E4FCFD120FD31218A5121937780A12D4
:100B7400110E9002E81217EE1218E0802A9002D4A7
:100B84001218ABAE0EAF0F1217B5C004C005C006E5
:100B9400C007AE0AAF0B1219301211401217B8D0A9
:100BA40003D002D001D000120FB8121893E50870D8
:100BB40003020D10121809C31210FD50739002D8CD
:100BC40012185A1217FDC006C007AE18AF19121832
:100BD40066D007D00612105E1218739002E012114C
:100BE40040AE1CAF1D1217F712186E9002D81218DF
:100BF4005A12189C121947C006C007AE18AF191232
:100C04001866D007D0061218999002E41218499079
:100C140002E4500B1211409002E41217C68007122E
:100C2400118D000000001218E6AE12AF13020CF48E
:100C3400121809D31210FD4012AE18AF191218661B
:100C440012192A120FC5121873800A9002E01211A9
:100C54008D00000000121803780A12112112187373
:100C640012194D50181218F7FEE4FCFD9002E4121C
:100C740018001218E612105E121873800A9002E42B
:100C840012118D000000009002E0121140AE1AAF64
:100C94001B1217F712186E1217D8C31210FD501A30
:100CA4009002D8121140C374FF9BFF74039AFEE4B0
:100CB40099FDE498FC12189C800A9002E412118DAC
:100CC400000000009002E412185A12189C12194DE8
:100CD4005017121947C006C0071218F7AB07FAE4F9
:100CE400F9F8D007D0061218991218E6AE1CAF1DF9
:100CF400E4FCFD120FD312189C121947780A121142
:100D04000E9002E41218001218E680279002D812FE
:100D140018ABAE12AF131217B5C004C005C006C09D
:100D240007AE1AAF1B12180D1217B8D003D002D099
:100D340001D000120FB812187390026E1211349081
:100D440002DC12183140111217F190026E1217EEE4
:100D5400121819900276801D9002761211349002B6
:100D6400DC12185050121217F19002761217EE127C
:100D7400183B90026E12118190027E12113490027F
:100D8400E0121831401112180390027E121800125A
:100D94001819900286801D9002861211349002E088
:100DA40012185050121218039002861218001218CA
:100DB4003B90027E12118190027612113412189324
:100DC4009002861211341218739002DC12182A4011
:100DD4000A9002DC12118D000003FF9002E0121849
:100DE4002A400A9002E012118D000003FFC284120F
:100DF40017F1780212110E900290EEF0A3EFF012A8
:100E040017F1EF5403FFE4FEFDFC7806121121C034
:100E140004C005C006C007121803780612110ED0CC
:100E240003D002D001D0001210F0900292EEF0A391
:100E3400EFF0121803EF543FFFE4FEFDFC780212BA
:0C0E44001121900294EEF0A3EFF0C2091F
:100E5000D007D006D005D004D003D002D001D000F6
:0B0E6000D0D0D082D083D0F0D0E032A0
:031A15000222D5D5
:1022D500C0E0C083C082C0D075D000C004C005C0B6
:1022E50006C007C2FF9002A2E004F0C36480948395
:1022F5005007E0FF3395E0801F9002A2E0FFC36422
:10230500809485502B9002A6E0FD3395E0FCEF33D9
:1023150095E0FEEF2DFFEE3CFEEF25E0FFEE33FEF0
:1023250074902FF58274023EF583A3E0F5A3801324
:102335009002A6E02402F0E0D3648094854002E494
:10234500F0D284D007D006D005D004D0D0D082D02A
:0423550083D0E0321F
:031A2D000225D9B6
:1025D900C0E0C0F0C083C082C0D075D000C000C0C8
:1025E90001C002C003C004C005C006C00753917FE3
:1025F900122359D007D006D005D004D003D002D079
:0E26090001D000D0D0D082D083D0F0D0E0320B
:031A2100021D663D
:101D6600C0E0C0F0C083C082C0D075D000C000C043
:071D760004C005C006C00710
:101D7D00C2EDAFBEEFFEADBDEDFF9002A4E070046D
:101D8D00A3E064027054E5BBB403047D0180027DC1
:101D9D0000E5BBB40D047C0180027C00EC4D603588
:101DAD00D3EF94C8EE648094834010AFBBEF25E071
:101DBD00244EF876030876C8021E43C3EF9468EEEE
:101DCD0064809480500FAFBBEF25E0244EF8760071
:101DDD0008766880611218BE805C1218BE9002A44D
:101DED00E475F001120F8CFEC3E5F0940AEE6480E9
:101DFD00948050099002A4A3E0F5BB803690028E2A
:101E0D00E475F001120F8CFED3E5F09413EE6480AF
:101E1D009480400B90028EE4F0A3740AF0D20E90E1
:101E2D0002A4E4F0A37402F0D20990028EA3E05450
:061E3D000FF5BB75E8D0B3
:101E4300D007D006D005D004D000D0D0D082D08324
:051E5300D0F0D0E032E8
:1028B600EFFD90033AE0FB3395E0FAC3EB9D74809D
:0428C600F86A9822F2
:081F3E00900335EFF0A3EDF074
:101F4600A2009204C2062017FDD217900339EBF0C7
:101F5600C201D202D2057F01C2C4C207D2C530C0B7
:101F6600FDE5C054F02480607624C0601B24E06048
:101F760003022005900339E0F5C2A201E43342C210
:101F8600C2C5E4A3F002200730C149300707D2C515
:101F9600C20702200730020CC202D203900336E0C9
:101FA600F5C2805D300311C203900335E0F5C230FF
:101FB600044FD207D20180492001461228B6500E9E
:101FC600900338E0F5C290033AE004F08033D2C4BF
:101FD600C217802D300504D2C58026D20680221273
:101FE60028B6500CA3E5C2F090033AE004F0D2C143
:101FF60090033AE0B5070AC217C2C1D2C48002D222
:102006000630060853C0BF43C040C217C2C03017CF
:0920160003021F6490033BE0FF8C
:01201F00229E
:101E580090390175F016ED1211BEEC75F016A42537
:101E680083AF8290030EF0A3EFF0900306E075F0C5
:101E780016A42401F9743935F0FA7BFF22E075F0D5
:101E8800169039011211BEAF82AE83229002C9E4C6
:101E980075F001020F8C9002ACE475F0011211CAC2
:101EA800AE02AF01227B007A007908900341E4F08A
:101EB800A322E024FFFFE434FFFE900307E0FCA325
:101EC800E0FD22AD04EDFFEEF0A3EFF090035B74AC
:101ED8000FF0229002C9E0FCA3E0FDC39416EC9435
:101EE8000022E475F001120FA285F082F583E493D5
:101EF8002224FFFEE434FF900307F0A3CEF02290E3
:101F0800030B1211E1E4900309F0A3F022E490021C
:101F1800C9F0A3F022AF05E4F0A3EFF0E07F00FEE4
:101F28002274B12DF582E43402F583229FEE648099
:061F3800F8EC6480982221
:1024AE009003547404F0E4A3F0A3F012295B7E3978
:1024BE007F007B017A037954121EB304F0122617A3
:1024CE00E4900355F0900355E0FFC3941E50187529
:1024DE00F016EF121E89121EAD7416F0122617900A
:1024EE000355E004F080DE7E3B7F957B017A037915
:0C24FE0056121EB304F012261702275DD0
:1028F10020180F300A083087071229638002D28717
:03290100D21822C7
:10280200903B95E493600C903900E4936404600378
:092812001224AEE490035BF022F5
:10284C0090035B121E7578087C007D007E007F165D
:06285C00120F3BC218221E
:1028770012295B90035B121E85121EAD7416F012AF
:05288700261702275D89
:061A1B00122877C2182218
:08202000900302EFF0A3EDF0C4
:10202800A2AFE433900310F0C2AF900302E0FFD3F5
:102038009B4033EF121EF9EB14900306F090030354
:10204800121EBAD3121F345058121E58121F0712EC
:1020580020B440FB12275D900307121E97900306D9
:10206800E004F0022045900303E0121EF9900305F6
:10207800E014A3F0900302121EBAC3121F344021C9
:10208800121E58121F071220B440FB12275D90033E
:102098000774FFF5F0120F8C900306E014F002208D
:0C20A8007C900310E024FF92AF02264F52
:1020B40090030BE475F0011211CAAE02AF01900354
:1020C4000EE475F001120FA285F082F583E493FD0E
:1020D4001223D8900309E475F001120F8CC3900306
:0B20E4000AE09416900309E09400222B
:0520EF009002ABEDF0D2
:1020F400A2AFE4339002CBF0C2AFEF149002C7F06A
:10210400EB14A3F09002ABE014FF9002C7E0D39F5E
:1021140040030221AEA3121E85121F15121EDB50AE
:10212400190FEFAA0670010E14F5828A83E493FB5B
:10213400121F29EBF0121E9480E29002C8121E7541
:102144009002AC1211E19002C7121E859002AFEE0C
:10215400F0A3EFF0121F15121E9E9002AF121EEA9A
:10216400FD1223D8121E94C39002CAE09416900262
:10217400C9E0940040E19002C7121E759002AC12AF
:1021840011E1121F15121EDB5010121E9E121F2980
:10219400E0FD1223D8121E9480EB12275D9002C733
:1021A400E004F0A3E004F00221089002CBE024FF55
:0521B40092AF02264F6E
:0722490090031CEBF0AC0751
:10225000A2AFE433900324F0C2AF90031D121F1D00
:1022600090031DF0A3EFF090031D121ECB12295B0B
:1022700090035B121E7590031F1211E1E49003227C
:10228000F090031DE0FCA3E0FFECFD90031CE0FBDD
:10229000E4900338F0D200121F3E900323EFF0FDCC
:1022A00090031F121EA11223D890031D121E979097
:1022B0000322E004F0E0C3941640C612275D9003A9
:1022C0005BE004F0E0C3941E40A3900324E024FFED
:0522D00092AF02264F51
:0721B900900325EBF0AC07D9
:1021C000A2AFE43390032CF0C2AF900328121F1D7E
:1021D000900328F0A3EFF0900328121ECB90035B2E
:1021E000E0FFC3941E505775F016EF121E8990033E
:1021F0002AEEF0A3EFF0E4900326F0A3F09003287A
:10220000E0FCA3E0FFECFD900325E0FB90032A1225
:102210001EEA900338F0C200121F3E900328121EDF
:1022200097900326121E97C3900327E094169003FD
:1022300026E0940040C790035BE004F0809F900389
:092240002CE024FF92AF02264FAE
:05278300900330EDF0B1
:1027880090033174FF12114EEC4D4E4F60109003C0
:0E27980030E0120F7A740129F9E43AFA80E277
:0127A6002210
:1027C900E475F001120FA285F082F5832275B7A591
:0F27D90075B7F18F828E8322EEF0A3EFF0A3226B
:10281B00A2AFE433FDC2AF758F031227D6E4F0F5F8
:08282B008FAF05EF24FF92AF0F
:012833002282
:1027E800A2AFE433FCC2AF758F011227D6EDF0E437
:0927F800F58FAF04EF24FF92AF4E
:0128010022B4
:102598009003501227E1ECF0A3EDF0EB4A60319084
:1025A8000350E0FEA3E0FFA3E0FCA3E0F5828C83E8
:1025B800E0FD1227E8EB1B70011A900352E475F056
:1025C80001120F8C900350E475F001120F8C80CB30
:0125D80022E0
:08295B00E4900000F0A3F0225B
:10275D00900000E0FEA3E0FF12281B900000E0FEB9
:10276D00A3E0FF7C007D027B007A02122598E490A5
:06277D000000F0A3F022B1
:0A23D800A90590034AEEF0A3EFF010
:1023E200EE54FEFE900000E0FCA3E0FD7002EE6CF5
:1023F2006044ED4C600312275D90034AE0FEEE5408
:10240200FEFE7F00900000F0A3EFF090034C122735
:10241200E17400F0A37402F07F007E0290034C127C
:1024220027C9E493FD90034E1227C9EDF0EF1F7008
:10243200011EEF4E70E690034AE0FCA3E0FDEC546F
:0E24420001FC74022DF58274003CF583E9F074
:012450002269
:1026170090033C1227E11211E190034174FFF5F09A
:10262700120FA245F0602090033CE475F001120FF1
:10263700A2AFF0FE90033EE475F0011211CA120F2B
:0826470061FD1223D880D222AC
:1019F200900357EFF0A3EDF07F0A122451900357A2
:101A0200E0FF122451900358E0FF12245102296B87
:082963007F0212245102296BCE
:06268300122972EF60272E
:102689009003597403F0A37443F012270D90035972
:10269900E475F001120FA285F082F583EFF012299B
:0726A90078EF70E67F0122CB
:0326B0007F002286
:10288C0090035CEFF07F2F12245190035CE0FF1259
:05289C00245102296B2C
:1028A10090035DEFF07F3012245190035DE0FF1241
:0528B100245102296B17
:02254E00C115B5
:1025510090020CE475F001120FA285F082F583223E
:10256100900208E0FFA3E0CF900204F0A3EFF02275
:1025710090020C7402F0A3743EF022900204E47500
:10258100F001120F8C7E027F6E900204E022EE9029
:072591000208F0A3EFF022A5
:0C292000758920438E08758DE8D28E2248
:1028CA0075C101E4F5C2F5C053C17F43C18043F627
:0428DA0001022920AE
:10264F007E027F0E900206EEF0A3EFF090020AEEEC
:10265F00F0A3EFF0900202EEF0A3EFF07E027F3EC8
:10266F0012258F90020CEEF0A3EFF0EE122569C247
:04267F00140228CA4F
:1027360090020A122554EFF090020A122554EDF089
:1027460090020AE0B4020FA3E0B43E0A90020A74B3
:0727560002F0A3740EF02253
:07296B00C214C2C4D2C52250
:1024510020142FD21412255174FFF07C027D6E904E
:10246100020CE0B50408A3E0B5050312257112259D
:1024710051E4F090020CE0B50408A3E0B5050312A5
:102481002571122551E4F090020CE0B40208A3E09A
:10249100B46E03122571122551EFF090020CE0B4D5
:0D24A1000208A3E0B46E031225717F012232
:1026E100900206E0FCA3E0FD900202E0B50408A31D
:1026F100E0B505037F0022900206E0FCA3E0F5822D
:0C2701008C83E0B507037F01227F0022DB
:10270D00900206E475F001120F8C9002061225540A
:10271D00E0FF900206E0B4020FA3E0B43E0A90027F
:08272D00067402F0A3740EF023
:012735002281
:062972007FFF1226E122A6
:06297800E4FF1226E1223B
:031A1800021A307F
:101A3000C0E0C0F0C083C082C0D075D000C000C07C
:101A400004C005C006C007E5C054FE1211EA1B9988
:101A5000081B990A1BAF0C1BAF0E1B72101B7212D6
:101A60001B8E141B8E161B651C1B651E1B61241B05
:101A700061261B24281B242A1B322C1B322E1ABC45
:101A8000C01AC6C21A8EE01A8EE200001BB8C2C588
:101A900012257CB5060BA3E0B507069002041225BB
:101AA00074900204122554E0F5C2900204E06E70B6
:101AB00003A3E06F6003021BB8021B1B122561D257
:101AC000C4D2C5021BB890020CE0FEA3E0FF900256
:101AD00004E0FCA3E0FDB5070EECB5060A12258F65
:101AE000C2C5D2C4021BB88D828C83E0B4FF03024E
:101AF0001BB412257CB5060BA3E0B50706900204C3
:101B0000122574900204122554E0F5C2900204E0FC
:101B10006E7003A3E06F6003021BB89002041225ED
:101B200074021BB8E5C260289002A9E065C260207B
:101B30008013122561C2C5D215E5C260139002A9B7
:101B4000E065C2600BC2C4C2C5C2C1C216021BB8E6
:101B5000ADC27FFF122736C2C4C2C5D2C1D2168021
:101B600057D2C58053900204E0FFA3E0CF12259026
:101B7000804690020AE0FFA3E0900202CFF0A3EFBC
:101B8000F0C2C4C2C1301530D2C5C215802A122598
:101B900061C2C4C2C1D2C5801FC2C4C2C52016045E
:101BA000C2C18014ADC2E4FF122736D2C18009122F
:101BB0002561C2C1C2C4D2C5C2C0D007D006D005FB
:0F1BC000D004D000D0D0D082D083D0F0D0E0328B
:10195700120FD3900318121181900311E025E02490
:101967000AF8E6FE08E6FF223395E0FDFC78101240
:101977001121900318121181900318229003141259
:101987001181E47FFF7EFFFDFC900314021140905C
:101997000311E0FF25E0243AF822EF25E0243AF886
:1019A70076000822900312E064809480229003015D
:1019B700E09F900300E09E90031822FAF9F8120FB7
:1019C700D390031802118190031402113425E024E7
:1019D700ECF582E43402F58322900318121134786F
:0B19E7001002110E900311E025E02219
:05150F00900311EFF054
:10151400C20F25E02426121968900300EEF0A3EF11
:10152400F0ED25E0244EF8E6FA08E6C39FFFEA9EB4
:10153400900312F0A3EFF030103EC31219AB502405
:10154400121996E6FA08E64A70051219A1760312F2
:10155400199608E616187001161486024A600302EA
:1015640015FA803FD3900313E094041219AB40059D
:10157400C2100215D90215F0D3900313E09400129F
:1015840019AB403E121996E6FA08E64A700512199C
:10159400A1760312199608E616187001161486022D
:1015A4004A70531219A17601ED25E0244EF8E6FCA9
:1015B40008E6FDEF25E02426F8A60408A605D20FC8
:1015C4008034C3900313E094FC900312E06480948D
:1015D4007F5019D210ED25E0244E1219681219EB30
:1015E4002426F8A60608A607D20F800A1219EB24AF
:1015F4003AF8E4F608F6E525452460030217952039
:101604000F03021795900311E0FD25E0240AF8E684
:10161400FE08E67806C333CE33CED8F9FFED1219AF
:10162400D4E04EFEA3E04FFFE4FCFD90031412113E
:1016340081900312E0FEA3E0FFD39400EE64809453
:101644008050030216CBEE12196F121134C006C07B
:1016540007900300E0FEA3E0FFC374FF9FFF740341
:101664009EAB07FAE4F9F8D007D00612105E1219FF
:1016740079121140C000121960C374FF9FFF7403F4
:101684009EFEE4FCFDD000121957D31219B4400891
:10169400121134E47B508006121134E47B301219A9
:1016A400C2121990C0001219E0D000120FB812191A
:1016B40083D31210FD500302175690031412118D98
:1016C4000000FFFF021756900312E0FEA3E0FFC3E1
:1016D400E49FFFE49EFE12196F121134C006C00786
:1016E400900300E0FEA3E0FBAA06E4F9F8D007D0DB
:1016F4000612105E121979121140C000121960E42A
:10170400FCFDD000121957C31219B4500812113439
:10171400E47B508006121134E47B301219C2121992
:10172400CEC004C005C006C0071219E0A804A9056C
:10173400AA06AB07D007D006D005D004120FC512F5
:101744001983D31210FD400A90031412118D000066
:1017540000001219CE900311E0FB1219D4EEF0A38D
:10176400EFF01219CE780612110E900314121181A3
:10177400EB121964E4FCFD121990C31210FD601100
:101784001219CE1219EB240AF8A60608A607122885
:01179400F163
:011795002231
:03000000020800F3
:03000300021A03DB
:03000B00021A06D0
:03001300021A09C5
:03001B00021A0CBA
:03002300021A0FAF
:03002B00021A12A4
:03003300021A1599
:03003B00021A188E
:03004300021A1B83
:03004B00021A1E78
:03005300021A216D
:03005B00021A2462
:03006300021A2757
:03006B00021A2A4C
:03007300021A2D41
:10080000E4F5D9E5EF7480F5FF7402F5EF787FE445
:10081000F6D8FD9000007F007E04E4F0A3DFFCDE4C
:07082000FA75817202086203
:10082700021BCFE493A3F8E493A34003F68001F2FD
:1008370008DFF48029E493A3F85407240CC8C333D2
:10084700C4540F4420C8834004F456800146F6DFA1
:10085700E4800B010204081020408090250AE47E02
:10086700019360BCA3FF543F30E509541FFEE49396
:10087700A360010ECF54C025E060A840B8E493A35D
:10088700FAE493A3F8E493A3C8C582C8CAC583CA88
:10089700F0A3C8C582C8CAC583CADFE9DEE780BE40
:01255000008A
:100E6B00E709F608DFFA8046E709F208DFFA803E69
:100E7B0088828C83E709F0A3DFFA8032E309F60856
:100E8B00DFFA8078E309F208DFFA807088828C83BE
:100E9B00E309F0A3DFFA806489828A83E0A3F60872
:100EAB00DFFA805889828A83E0A3F208DFFA804C4C
:100EBB0080D280FA80C680D4806980F28033801023
:100ECB0080A680EA809A80A880DA80E280CA80338C
:100EDB0089828A83ECFAE493A3C8C582C8CCC58304
:100EEB00CCF0A3C8C582C8CCC583CCDFE9DEE780D4
:100EFB000D89828A83E493A3F608DFF9ECFAA9F053
:100F0B00EDFB2289828A83ECFAE0A3C8C582C8CCA8
:100F1B00C583CCF0A3C8C582C8CCC583CCDFEADEC1
:100F2B00E880DB89828A83E493A3F208DFF980CC23
:100F3B0088F0EF60010E4E60C388F0ED2402B4041C
:100F4B000050B9F582EB2402B4040050AF232345C3
:060F5B008223900EBB731F
:100F6100BB010689828A83E0225002E722BBFE028E
:090F7100E32289828A83E49322C1
:100F7A00BB010689828A83F0225002F722BBFE0156
:020F8A00F32250
:100F8C00C5F0F8A3E028F0C5F0F8E58215827002F0
:060F9C001583E038F0228D
:100FA200A3F8E0C5F025F0F0E58215827002158302
:060FB200E0C838F0E8225F
:0D0FB800EF2BFFEE3AFEED39FDEC38FC2288
:0E0FC500C3EF9BFFEE9AFEED99FDEC98FC2227
:100FD300E88FF0A4CC8BF0A42CFCE98EF0A42CFCBD
:100FE3008AF0EDA42CFCEA8EF0A4CDA8F08BF0A43B
:100FF3002DCC3825F0FDE98FF0A42CCD35F0FCEB9A
:101003008EF0A4FEA9F0EB8FF0A4CFC5F02ECD395E
:0F101300FEE43CFCEAA42DCE35F0FDE43CFC22CB
:1010220075F008758200EF2FFFEE33FECD33CDCC85
:1010320033CCC58233C5829BED9AEC99E582984008
:101042000CF582EE9BFEED9AFDEC99FC0FD5F0D6E5
:10105200E4CEFBE4CDFAE4CCF9A88222B800C1B90F
:101062000059BA002DEC8BF084CFCECDFCE5F0CB4D
:10107200F97818EF2FFFEE33FEED33FDEC33FCEB86
:1010820033FB10D703994004EB99FB0FD8E5E4F941
:10109200FA227818EF2FFFEE33FEED33FDEC33FC2E
:1010A200C933C910D7059BE99A4007EC9BFCE99A22
:1010B200F90FD8E0E4C9FAE4CCFB2275F010EF2F67
:1010C200FFEE33FEED33FDCC33CCC833C810D70767
:1010D2009BEC9AE899400AED9BFDEC9AFCE899F8A2
:0E10E2000FD5F0DAE4CDFBE4CCFAE4C8F92235
:0D10F000EF4BFFEE4AFEED49FDEC48FC22FF
:1010FD00EB9FF5F0EA9E42F0E99D42F0E89C45F049
:01110D0022BF
:10110E00E8600FECC313FCED13FDEE13FEEF13FFBF
:03111E00D8F122E3
:10112100E8600FEFC333FFEE33FEED33FDEC33FC2C
:03113100D8F122D0
:0C113400E0FCA3E0FDA3E0FEA3E0FF222E
:0C114000E0F8A3E0F9A3E0FAA3E0FB2232
:10114C007401FF3395E0FEFDFCA3A3A3E0CF2FF0C9
:10115C00E582158270021583E0CE3EF0E5821582A1
:10116C0070021583E0CD3DF0E58215827002158387
:05117C00E0CC3CF02274
:0C118100ECF0A3EDF0A3EEF0A3EFF022E1
:10118D00A8828583F0D083D0821211A41211A412EB
:10119D0011A41211A4E473E493A3C583C5F0C58310
:1011AD00C8C582C8F0A3C583C5F0C583C8C582C8AC
:0111BD00220F
:0C11BE00A42582F582E5F03583F583223C
:1011CA00F8E0FBA3A3E0F925F0F0E58215827002AE
:0711DA001583E0FA38F02252
:0911E100EBF0A3EAF0A3E9F0220F
:1011EA00D083D082F8E4937012740193700DA3A394
:1011FA0093F8740193F5828883E4737402936860A8
:06120A00EFA3A3A380DFA7
:00000001FF
